:100000000019002031090000234600001D090000EE
:100010001D0900001D0900001D090000000000006E
:10002000000000000000000000000000E50A0000E1
:100030001D09000000000000B10A00001D090000B9
:10004000710C0000710C0000710C0000710C0000BC
:10005000710C0000710C0000710C0000710C0000AC
:10006000710C0000710C0000710C0000710C00009C
:10007000710C0000710C0000710C0000710C00008C
:10008000710C0000710C0000710C0000710C00007C
:10009000710C0000710C0000710C0000710C00006C
:1000A000710C0000710C0000710C0000710C00005C
:1000B000710C0000710C0000710C0000710C00004C
:1000C000710C0000710C0000710C0000710C00003C
:1000D000710C0000710C0000710C0000710C00002C
:1000E000710C0000710C0000710C0000710C00001C
:1000F000710C0000710C0000710C0000710C00000C
:10010000F8B5174D284604F0ABFC044628B32A691D
:10011000A968136843F0400313600B68114A062175
:1001200028469847002818DB0F4F104EAB68402137
:100130005B692846984700280FDB84F0010414F01F
:10014000FF0414BF39463146094803F029FE002157
:100150004FF4004003F030FAE8E70020F8BD00BF9C
:10016000E84E0000010006007052000073520000CB
:1001700077520000014B1B68184700BF00000020A9
:10018000014B1860704700BF0000002030B585B0FB
:1001900004460D4610220021684604F0EFFD0223BC
:1001A0008DF802302A46044B01932146684603F03D
:1001B00009FE05B030BD00BF7501000080B50546E1
:1001C0000E461746984603F015FA034604F042FE21
:1001D000DFF81890044649F8003042463046394668
:1001E000A84754F8090000F011FC00BF0800000007
:1001F0002DE9F047058B04462807904611D40229C3
:1002000005F0070540F0CC80204604F027F978B1CE
:100210000138218B042811D8DFE800F0C2106D8569
:10022000950001290CBF45F0100545F020052583F8
:1002300088F31188BFF36F8FBDE8F08701F0070ADC
:10024000AA4500F0A5800027B9463E46A368002BCA
:1002500000F0BC8041F00801218388F31188BFF3CE
:100260006F8FA168002900F0BA800D68002900F0A6
:10027000B680D1F80480334652462046C047002D50
:1002800076D02B6829461D46F0E701F007035A1F78
:10029000012A1BD8002221F00701062B276889B20A
:1002A000C4E9002209D13B4603E0628B013262833C
:1002B0001B68002BF9D141F002012183204604F094
:1002C000CDF800287AD041F0200176E0042B0AD145
:1002D00021F0070189B22183204604F0BFF810B154
:1002E00041F020012183218B01F0070AAA454FD05C
:1002F0000027B946AAE7236921F0070141F006016A
:10030000062DD3F8009021832DD1B9F1000F3FD0F5
:1003100041F00801218388F31188BFF36F8F3A49B8
:100320002046C84729E021F00701236941F0040174
:1003300089B2042DD3F804902183E6D000273E46ED
:100340004FF0040A82E721F00701236941F005011B
:1003500089B2052DD3F808902183D6D000273E46D8
:100360004FF0050A72E700273E464FF0060A6DE798
:100370002B4687E7B9F1000FD1D1EFF31188202385
:1003800083F31288BFF36F8F238B23F0080323833B
:10039000258BEA062ED525F01003238305F00705EB
:1003A0006669218B002EBFF670AF00232768C4E971
:1003B000003321F0070141F001012183218B01F07D
:1003C000070AAA454FF000097FF440AF002F9CD0E8
:1003D00041F00801218388F31188BFF36F8F002F4C
:1003E000C8D03D68394633465246204604F062F88C
:1003F0002F46F4E7AB067FF51BAF25F020032383E0
:1004000005F0070500E700BFE1440000014B036071
:10041000002070479850000008B5044804F011F817
:10042000BDE80840024804F00CB800BF8652000046
:10043000BB520000014803F00BBB00BF9850000006
:1004400038B5044618B90F4B0F485B689847616888
:10045000B1F5683F10D0B1F5680F0DD00B4DA94232
:100460000AD011F46861206807D00146084804F0FA
:1004700052FB00232360656038BD142204F07EFC2B
:10048000F9E700BFC4000020E95200002C5F5CA91E
:100490004008002008B520B34368B3F5683F10D189
:1004A00001220368BFF35B8F53E8001F002903D1CB
:1004B00043E800200028F7D1BFF35B8F0DD1002067
:1004C00008BD094A93420AD000684FF0FF324FF04E
:1004D000FF3302F0A3FC0028F1D00448F0E7044801
:1004E000EEE76FF4E040EBE72C5F5CA9E98FFFFFDC
:1004F000EA8FFFFF08B5D8B14368B3F5683F10D164
:1005000000220368BFF35B8F53E8001F012903D16A
:1005100043E800200028F7D1BFF35B8F0BD1002008
:1005200008BD074A934208D0006802F0EFFCF6E7E6
:100530006FF4E040F4E70348F2E70348F0E700BF58
:100540002C5F5CA9E98FFFFFEA8FFFFF10B504461F
:1005500018B91D4B1D485B6898476368B3F5683F41
:100560002FD0B3F5680F2CD0194A934219D12368C4
:1005700003BB18484FF0FF324FF0FF33214602F023
:100580001FFC08B923681BB90F4B13485B689847D9
:1005900020681422002104F0F1FB4FF468636360CB
:1005A00008E0B3F5683F0DD83A2B03D040F6BA62A5
:1005B0009342DED1206804F0E6FA636843F03A0320
:1005C000636010BD054AF3E7C4000020E952000053
:1005D0002C5F5CA9400800200F5300003A00003A4D
:1005E00008B5064906484023142204F086FABDE8FF
:1005F00008400449044803F09DBA00BF40030020AE
:1006000040080020A0500000B450000030BFFFF7A9
:10061000FDBF00BF2DE9F0410B4EDFF8308006EB47
:100620000807CC1B054632460949204604F098FBD2
:10063000A01942460021083C04F0A0FB2C6707F1FA
:100640000800BDE8F08100BF0000000004000000C9
:1006500090500000074A936893F90E10002907DBB9
:10066000526993421FBF044A536843F0805353605A
:10067000704700BF1C09002000ED00E070B5264B5C
:1006800015469A6A12F0100F9A6A14BF11241024AA
:1006900012F0080F9A6A18BF1224920706460AD56C
:1006A000586B9A6A140634D519B19A6A22F08002FE
:1006B0009A62132401E06FF01500174B9A6A12F04A
:1006C000010F9A6A18BF142412F0200F9A6A18BFFB
:1006D0001524D20602D49B6A9B070AD50E4B5B6891
:1006E000190506D5314600F079FA10B180F3098872
:1006F0000224094B9A6A920642BF5A6A22F40052B7
:100700005A629A6A42F0FF029A6200232B702046D6
:1007100070BD6FF01500CCE700ED00E0134B9A6A56
:1007200012F0007F9A6A14BF1E201D2012F0807FF5
:100730009A6A18BF1F2012F4002F9A6A18BF21204E
:1007400012F4802F9A6A18BF222012F4003F9A6A8E
:1007500018BF232012F4803F9A6A6FEA02426FEAC0
:1007600012429A6218BF2420704700BF00ED00E0DB
:1007700010B5194B0246986A9C6A10F4805F14BF4A
:100780001720162014F4006F9C6A18BF1820A405C7
:1007900009D5986B986A000404D51AB19A6A22F4B4
:1007A00000429A6219200C4B9A6A12F4806F9A6A7E
:1007B00018BF1A20D2050CD49B6A13F4005F18BF2F
:1007C0001C20054A936A43F47F43936200230B7015
:1007D00010BD1B20F5E700BF00ED00E0F0B5484B71
:1007E0005B688BB00446C3F30803002585F31188CA
:1007F000BFF36F8F02F07F40B0F17F4F11D102F055
:100800000C0008280DD010074CBF0C460125002213
:10081000033B8DF80720032B05D8DFE803F02463A2
:1008200067602C46F3E700239DF80720CAB902AEA3
:1008300004F1200720686168324603C20834BC42D4
:100840001646F7D1099A002D54D0C2F3080121B9F8
:100850006FEA52226FEA4222099202A9184603F077
:10086000D6FE0BB0F0BD264BDA6A9107DBD4DA6A0C
:10087000002AD8DBDA6A5200D5D55A69A16942F458
:1008800080725A61BFF34F8FBFF36F8F5A6931F88F
:10089000021C22F480725A61BFF34F8FBFF36F8F37
:1008A0004DF6027291420AD09A6AD2B24AB10DF163
:1008B000070201212046FFF7E1FE0346B4E7236863
:1008C000B2E79A6A12F47F4F05D00DF107010120BB
:1008D000FFF74EFFF1E79B6AB3F5803FA3D3FFF725
:1008E0001DFFEAE70DF107020021E3E70DF1070123
:1008F0000020EDE722F4FF7222F00102ACE700BF16
:1009000000ED00E0044B5A6942F010025A615A6946
:1009100022F008025A61704700ED00E0EFF3088012
:10092000EFF3098101B57246FFF758FF01BD00BF23
:10093000002080F31488BFF36F8F01F0BDFA002010
:100940000D490860BFF34F8F0C4880F3088800F012
:100950002BF8202080F3118809484FF404614018D7
:1009600080F30988EFF314800221084380F3148890
:10097000BFF36F8F00F0FAF894ED00E0001900204B
:10098000400B00200749D1F890200023C2F3072232
:100990001846934200DB7047C1F89830C1F8A000B8
:1009A0000133F6E700ED00E008B572B6002383F3EB
:1009B0001388FFF7E7FF144B4FF0FF32C3F8802096
:1009C000C3F88420C3F88820C3F88C20C3F8902093
:1009D000C3F89420C3F89820C3F89C20C3F8802162
:1009E000C3F88421C3F88821C3F88C21C3F890216F
:1009F000C3F89421C3F89821C3F89C2162B6BFF3D1
:100A00004F8FBFF36F8F08BD00E100E0084B9B687C
:100A100083420BD1EFF3058343B1064B5A6842F092
:100A200080525A605A6A22F400425A6204F05DB958
:100A30001C09002000ED00E0094A93686FF00A01EC
:100A40009967084958674B6843F080534B6000230F
:100A500083F31188BFF36F8F9368986F704700BF5F
:100A60001C09002000ED00E010B50446EFF31183EF
:100A7000202383F31288BFF36F8F0A4B5869986065
:100A8000094B4FF000625A60084B026F1A60002257
:100A9000436F426783F31188BFF36F8F00F006F94D
:100AA000204610BD1C09002000ED00E05C0800207D
:100AB0000B498A684FF030001044EFF3098C80E84E
:100AC000F01F74467046FFF7CFFFA64604498A68B8
:100AD00002F1300090E8F01F8CF3098870470000A5
:100AE0001C0900201EF0040F0CBFEFF30880EFF389
:100AF0000980816911F8021C0229FFD001B503F0B9
:100B00008CFD01BD40B2002807DB044A41090123E6
:100B100000F01F00834042F82130704700E100E000
:100B2000054B420900F01F0053F82220012303FA6D
:100B300000F01040704700BF00E100E040B2002824
:100B4000A8BF00F1604001F10101B8BF064B4FEAB8
:100B50004111ACBF00F5614000F00F00C9B2B4BF55
:100B6000195480F80013704714ED00E00B4A08B5E3
:100B70000B4B22F07F029A60BFF34F8FBFF36F8F52
:100B8000D3F8882022F47002C3F8882002F054F8C9
:100B900002F0BCFD00F060F802F092F800000000E6
:100BA00000ED00E042F8203C009B42F81C3C0A4962
:100BB000019B42F8183C029B42F8143C21F00101D1
:100BC0004FF0807342F8043C42F8081C0023203A9E
:100BD00002654367704700BFBD010000094A034634
:100BE000906870B113F1160F006E05D0A0F14002AD
:100BF0009A4205D8834203D2814228BF0020704721
:100C0000002070471C09002008B515460B4A0C4B04
:100C10009060026F1A600E4600F048F82C4686F38A
:100C200009884FF00000074B984720464FF000011D
:100C30004FF000024FF00003034C20471C09002036
:100C40005C08002039460000BD010000014B102265
:100C50001A61704700ED00E0044800232021C2180B
:100C60000133302B82F80013F9D1704700E100E026
:100C700008B5EFF30583064A103B02EBC30152F8B7
:100C8000330049688847BDE80840FFF7E3BC00BF70
:100C9000104F0000024B034A0348012100F076B8D0
:100CA0000000042000000020C4500000026E054B2C
:100CB000403A1A60044A4021C3E901121846012152
:100CC00000F06EB86008002000000B15084AC2F85A
:100CD00098000B6823F01F03034343F01003C2F88E
:100CE0009C308B6843F00103C2F8A030704700BF0E
:100CF00000ED00E02DE9F043DFF8608085B00E469E
:100D00001F4604464FF00009B14523DA6068D8B1A8
:100D10003FB1411E08421BD11F2819D9236819422F
:100D200016D12368019303F0AAFCA368034303933D
:100D3000D8F89050C5F30725D0B2013DA84207D896
:100D400001A9FFF7C3FF421C09F101090C34DBE7DD
:100D50006FF01502104605B0BDE8F08300ED00E02D
:100D6000044B0522C3F89420BFF34F8FBFF36F8F5E
:100D7000704700BF00ED00E0BFF35F8F024B002221
:100D8000C3F89420704700BF00ED00E010B5034C9D
:100D900001232278FFF7AEFF207010BD240B002046
:100DA00008B50B4A00231278FFF7A4FF10F1160FC5
:100DB00007D0084A0021D2F89030C3F307239842A5
:100DC00000DB08BDC2F89800C2F8A0100130F2E7BD
:100DD000240B002000ED00E02DE9F043534B544C70
:100DE000D3F890302568C3F307239D4285B000F205
:100DF0009A80FFF7C1FF00200C2685421AD14D4C86
:100E00004D4F25706846FFF701FBDFF82081DFF8C2
:100E10002C9106460025AE4213D123784349002089
:100E2000D1F89020C2F30722934276DBFFF798FFB8
:100E3000002042E0616806FB0011FFF747FF013028
:100E4000DBE7009800EB05114FEA051CCB683B403F
:100E5000B3F5000F48D00AD8B3F5001F30D0B3F572
:100E6000800F36D0B3F5801F10D00135D3E7B3F132
:100E7000807F42D0B3F1007FF7D150F80C30886802
:100E80004A6803F0FCFB40F4802009E050F80C3085
:100E900088684A6803F0F3FB40F0885040F4302043
:100EA000CDE901230390D8F890302078C3F30723CD
:100EB000013B98422AD96FF0150005B0BDE8F083D8
:100EC00050F80C3088684A6803F0D9FB40EA090002
:100ED000E6E750F80C3088684A6803F0D0FB40F031
:100EE000E06040F40030DBE750F80C3088684A6876
:100EF00003F0C5FB40F08270D2E750F80C308868F0
:100F00004A6803F0BCFB40F08870C9E701A9FFF70D
:100F1000DDFE237801332370A7E7C1F89830C1F8CC
:100F2000A00001337CE74FF0FF30C6E700ED00E0A2
:100F3000D0500000240B00200000F0FF000008113A
:100F400008B5024B1B689847002008BD6C080020BC
:100F5000034B044A1860937843F002039370704780
:100F60006C0800202400002008B50649064821F03E
:100F70000701C1F1005202F5802203F008FA0020B7
:100F800008BD00BF47190020700800200E4A012349
:100F9000C2F840354FF080424FF08051C2F87835AA
:100FA000D1F83001082808D1D1F83411052904D826
:100FB0000648415C09B1C2F838364FF0804301223F
:100FC000C3F880250020704700E001404B5300002B
:100FD00020B1034B800143F001031847704700BF65
:100FE000905000004FF08043D3F84036DB072ED5F9
:100FF0004FF01023D3F8043303F00703072B26D157
:10100000144A0123C2F80435D2F80034002BFBD077
:101010004FF01021D1F8043323F0070343F0040309
:10102000C1F804330023C2F804350A4AD2F8003468
:10103000002BFBD0BFF34F8F0749084BCA6802F45F
:10104000E0621343CB60BFF34F8F00BFFDE700208A
:10105000704700BF00E0014000ED00E00400FA0529
:10106000084B70B5C31A0D4607499B1004465943F7
:101070000648402203F021FB2B4601462046BDE8EE
:101080007040184790080020B76DDBB6C04E0000D6
:1010900073B50C4C0C4A4023041B00930D460B46C1
:1010A0000A49A41061430646094803F032FB011EB9
:1010B00005DA30462B4602B0BDE87040184702B052
:1010C00070BD00BF900800207D470000B76DDBB603
:1010D000C04E000010B5EFF31184202383F3128873
:1010E000BFF36F8F074A136823F00201DB0711601B
:1010F00002D4012003F02DFC84F31188BFF36F8F1D
:1011000010BD00BFE0080020002270B50121044698
:101110001046FFF713FD0F4801F05EF80E4B9842A2
:1011200015D101F069F826690C49304603F0E5F95C
:1011300000280BDB012535642469084904F11C00F3
:1011400003F0DBF9002801DBE564002070BD6FF0DF
:101150000400FBE7591200000000AD0BF450000042
:101160001FB500220123CDE90223094ACDF800D0A2
:101170006B46CDF804D003F0FAFA002805DB4FF4F3
:1011800080420023684601F021FF05B05DF804FBB2
:101190009B47000030B4104B0C2202FB0033014689
:1011A0000020D3E90E529863EFF31180202484F3DA
:1011B0001288BFF36F8F1C6C04F0C00444F002046B
:1011C0001C6480F31188BFF36F8F1DB12B46034859
:1011D00030BC184730BC704790080020C04E00005B
:1011E00010B4EFF31182202383F31288BFF36F8FC3
:1011F0001748016841F002040460C80707D482F36D
:101200001188BFF36F8F012010BC01F007B84FF0B9
:101210008041D1F80C04D1F80C14C907EFD5EFF3D5
:10122000118083F31288BFF36F8F0A490B6C03F0B0
:10123000C00343F002030B6480F31188BFF36F8F88
:1012400082F31188BFF36F8F002010BCFFF7A2BF9D
:10125000E00800209008002010B1012804D0704759
:10126000034B1B6C5B0701D1FFF794BF704700BFB6
:10127000900800202DE9F0413849BFF35B8F074605
:10128000012251E8003F41E800200028F9D1BFF3D6
:101290005B8F33B9324933484B60CB608A6003F0CF
:1012A0003FF97B1E012B2BD8012F07D14FF0804334
:1012B000D3F81C3403F00303012B21D003F06AFCA4
:1012C0000546F8B9284B1B78E3B14FF08043022262
:1012D000C3F808230646DFF894804FF08044D4F822
:1012E0001824D4F81834D20315D503F00303012BC6
:1012F00001D0012F0FD155B386F31188BFF36F8F43
:10130000BDE8F081EFF31186202383F31288BFF349
:101310006F8F0125DFE7ADB1304603F0A1F9D4F8B6
:101320001835002BDBD1D4F80421002AD7D0C4F81B
:101330000431D4F804310123C4F81835C8F88031D9
:10134000A360CCE70021212002F036F9E7E74FF057
:1013500080430222C3F80423D2E700BF8C08002098
:101360007C080020AC080020270B002000E100E0F2
:1013700008B5074803F074FB38B10648FFF7E8FDED
:101380000448FEF7FDFE002008BD6FF01200FBE7E9
:10139000FC4E0000991300000A2838B5074D04469A
:1013A00004D1AB680D215B6828469847AB680348B9
:1013B0005B68E1B29847204638BD00BFFC4E000094
:1013C000F0B54068057B01F01F0444EA4514056947
:1013D00087B0002D64D0B2F5001F00F1100506D1D2
:1013E0002146284603F035FB002007B0F0BD01AED2
:1013F0000027B2F5800F0197776039D1B3F1007FF4
:1014000014BF052304238DF804300023CDE90463C1
:101410000393836823FA01F111F001011AD1B2F1AB
:10142000A07F17D104F01F03620903F5E0732AD0EF
:10143000012A3BD11F4A52F82330DB070AD40DF1B1
:10144000030632462146284601F0C6F91A4B984257
:101450001CD0029603AA2146284601F07FF8174BBC
:10146000984220D101222146284601F019FABBE713
:10147000B3F1C06F05D0B3F1007F14BF0123022385
:10148000C1E70323BFE74FF0A042D4E73146284627
:1014900001F000FA094B9842DBD06FF00B00A4E793
:1014A0006FF08500A1E76FF015009EE751F823303B
:1014B000FFDE00BF000300500400AD0B0000AD0BC9
:1014C00038B545682B69B3B11035284601F0D2F91B
:1014D000044680B90146284601F098F9084B984225
:1014E0000BD108492246284601F070F92246052111
:1014F0000620FFF723FB002038BD6FF00400FBE758
:101500000000AD0B09150000420970B5034602D07A
:10151000012A17D070BD0D4E326951680029F9D0EB
:1015200003F01F0301250C689D400029F2D08A6852
:101530002A4002D04B68304698472CB12368214698
:101540001C46F2E7024EE7E72346F8E7E84E0000C4
:10155000D44E00002DE9F043466840F20635D0062F
:10156000337B87B002EA050554BFC2F34010032065
:1015700001F01F07B5F5837F144647EA43178DF83E
:10158000030045D00FD8062D18D007D8B5B1022DCD
:1015900040D06FF0150007B0BDE8F083B5F5807F4F
:1015A000F7D101250AE040F20222954234D0B5F588
:1015B000407F33D0B5F5007FEBD102250123220314
:1015C00003FA01F12CD57368C3F80815326982BBA0
:1015D00007F01F037F0929D0012F77D13E4A02EB84
:1015E000830284F48033D2F80017C3F30043C4F3BA
:1015F000404444EA430421F4E16144EA800421F0D8
:10160000070144EA05230B43C2F800370020C2E774
:101610000725D3E70425D1E70525CFE70325CDE747
:10162000630344BF7368C3F80C15CFE74FF0A042C3
:10163000D5E710360DF102023946304601F0CCF8FC
:1016400014F4403F80460CD13946304603F0FFF990
:10165000224B9845DAD19DF80210304601F014F97A
:10166000D4E701AB4FF0000903AA39463046CDE973
:101670000439CDE90199CDF80C9000F06FFF174BBC
:10168000984286D114F4003315D09DF803308DF8BC
:101690000E3084F48034C4F300444B4603AA394628
:1016A00030468DF80C508DF80D4001F011F80B4BC1
:1016B0009842CDD06DE7CDE9043303AA0DF10303C1
:1016C00039463046039300F049FFF0E703F5E07335
:1016D00052F82330FFDE00BF000300500000AD0BC6
:1016E000036803F01F025B09026004D0012B03486A
:1016F00018BF002070474FF0A04070470003005013
:101700002DE9F04FDFF86091DFF860A185B0154654
:10171000834600EB810140F2FF18594503D10020B8
:1017200005B0BDE8F08FDBF800305804C3F3C322E6
:10173000C3F3080400F191801B0E19F802704445B0
:1017400008BF4FF0FF34192B00F28A80DFE803F066
:101750000D141A1D20261D8888888836638888887D
:10176000888888888888667C7F82C5F80C45621CDA
:101770005ED10BF1040BD0E7C5F81445631CF8D01B
:1017800000265FE0C5F80845F1E7C5F81045F5E724
:10179000661CC5F80845ECD0002604E0601CC5F8BE
:1017A0000C45E6D0012603A80394FFF799FF039B9D
:1017B000012202FA03F3C0F80C3508E0C5F8084529
:1017C000002FDBD1631CD4D0002632460627DBF87D
:1017D0000030019303F40040002818BF002203A842
:1017E000009218BF01260394FFF77AFF039C019B28
:1017F000009A00EB8400C3F3412CD0F800473B0271
:1018000043EA8C03134304EA0A04234343EA4603EE
:10181000C0F80037ADE7C5F80C45D1E7C5F860451D
:10182000621CDBF80030A4D0C3F30043002BB9D016
:1018300003A80394FFF754FF039B012606FA03F362
:10184000C0F808353246C2E7C5F86445E8E7C5F890
:101850006845E5E7C5F86C45E2E76FF015005FE71E
:101860006FF085005CE700BF7C530000F0F8FCFFE0
:101870002DE9F041044647680D4603F08BF94FF01F
:10188000200888B9264B1B7873B16426606803F082
:1018900009F8F0B9012003F04EF8013EF6D100211D
:1018A000212001F089FEF0E7EFF31186314688F33D
:1018B0001288BFF36F8F606802F0F4FFA8B986F357
:1018C0001188BFF36F8FEFE786F31188BFF36F8F37
:1018D000E5E7EFF31186314688F31288BFF36F8F87
:1018E000606802F0DFFF0028EED0BB691D706368FE
:1018F000BA691B680020C3F844250122C3F84825B3
:10190000C3F82001D3F82041C3F85801D3F8580197
:101910009A6081F31188BFF36F8FBDE8F08100BF3B
:10192000270B0020F7B50546002201210220FFF712
:1019300005F90220FFF7E6F86A6811681369C1F833
:101940002435137D507D927D03431343C1F86C35DC
:101950006E68D6E9004313F0010348D02F6907F100
:10196000080002F0F4FF304B98425AD1387A04F163
:101970000C0204F5907102F0E0FF387A012707FAB3
:1019800000F000F0C1FB0823C4F80035B369C4F8C7
:1019900044350023C4F84835A760D4F85831002BEB
:1019A000FBD00021C4F800156B68DC6801AA204652
:1019B00002F04BFF002805DB019B226819791868AB
:1019C000FFF79EFE6A6813680821C3F80015117AB4
:1019D00051B9D269C3F834250122C3F83825C3F8B8
:1019E0001011D3F810111A60002003B0F0BD0822C6
:1019F000C4F80025B269C4F84425C4F84835012369
:101A0000A360D4F82031002BFBD00023C4F8203190
:101A1000D4F820310123E3604FF48073C4F8043319
:101A2000BBE76FF00400E0E70000AD0B70B50123E9
:101A300083400E4ABFF35B8FDC4352E8001F01EA8C
:101A4000040542E80056002EF7D1BFF35B8F4FF438
:101A5000803282400648C0F80823BFF35F8FBFF38F
:101A60006F8F0B4214BF0120002070BD0C090020B5
:101A70000010014070B40E49D1E90034D01AC318E7
:101A800044F1000422F07F46C1E90034A6F50013BA
:101A9000B3F5400F09D2074B1B681A0A1B069C19A5
:101AA000054B42F10005C3E9004570BC01F008BFD9
:101AB00090010020100900209801002011B3BFF30D
:101AC0005B8F0123104A834052E800CF4CEA030C9D
:101AD00042E800C10029F7D1BFF35B8F0B4A4FF4F6
:101AE00080338340C2F80433094BBFF35B8F1B681C
:101AF000BFF35B8FC340DB0742BF064B4FF400329E
:101B0000C3F80021704700BF0C09002000100140FD
:101B10000809002000E100E00D4B1868010A0006EA
:101B2000BFF35F8F0B4BD3F80435181841F1000158
:101B3000B3F5801F0AD2084BD3E90023904271EB22
:101B4000030303D210F1807041F10001704700BF20
:101B50001009002000100140980100202DE9F04FED
:101B600085B016461F469DF840A00446FFF75EFF6D
:101B70000190FFF7D1FFB04271EB070354D23E4B07
:101B8000301A67EB0101984271F100014FD23B4BD3
:101B900003EB0413D3E902239F4208BF96425ED0B1
:101BA00037494FF4803804F1500508FA04F8AD00C5
:101BB000C1F848832046ADB202F0A5FE26F07F4B67
:101BC00005F1804504F5A87305F58835DC464FF02E
:101BD00003090293029A2CF07F4341F82230C1F8A6
:101BE0004483D1F80435274A6FF00200C01A6044DC
:101BF00020F07F40904232D9286868B1D1F804358E
:101C00000393A3EB0B0020F07F40B0F5000F26D923
:101C1000204602F078FE039BBAF1000F07D109EBD2
:101C2000030C09F10109D5E7BAF1000F09D06FF0F3
:101C3000150520460199FFF741FF284605B0BDE88C
:101C4000F08F0123104ABFF35B8FA34052E8000FCF
:101C5000184342E800010029F8D1BFF35B8F074920
:101C60000E98230101EB0412C8500F9B5360C2E988
:101C700002670025DDE700BF010080008001002031
:101C800000100140FDFF7F00080900207FB51C4CBB
:101C90001C4BC4F80833C4F848331B4B00254FF0E5
:101CA000FF304FF0FF31C4F80855C3E902014FF48B
:101CB0008033C4F80433154B02264FF4003201215F
:101CC000C4F804631120C3F880212A46FEF736FFCA
:101CD0001120FEF717FF0E4A0123A3602360136053
:101CE0000C4B0D4A0093CDE9015500232846FFF720
:101CF00035FF3046FFF7BEFA284604B070BD00BF7E
:101D00000010014003000F008001002000E100E00E
:101D10000C090020751A0000FFFF7F002DE9F74332
:101D20002F4CD4F8043399070BD5D4F8043143B1C0
:101D30002C4A0023C4F80431D4F804311368013369
:101D40001360D4F80433DA0329D5BFF35B8F264B35
:101D500053E8002F22F0010143E800100028F7D1DA
:101D6000BFF35B8FD30702D4D4F84031BBB1002559
:101D7000C4F84051D4F84031FFF7CEFEEFF31182A2
:101D8000202383F31288BFF36F8F184BD3E90267C8
:101D9000B042B94106D282F31188BFF36F8F03B00E
:101DA000BDE8F0834FF0FF384FF0FF39C3E90289F7
:101DB000D3E900101D604FF48033C4F84833C4F8F1
:101DC0004051D4F8403182F31188BFF36F8F00295E
:101DD000E5D0009032463B4628468847DFE700BF03
:101DE0000010014010090020080900208001002097
:101DF00030B5431C124C85B005D08442A8BF0446C0
:101E0000012CB8BF0124FFF787FE0E4B0C4DD3E920
:101E10000013401AB0F5000F10D22218AA4228BFB2
:101E20002A4652184FF0000007490091CDE9010001
:101E300043F10003FFF792FE05B030BD2A46F0E7FC
:101E4000FFFF7F0090010020751A000008B5FFF722
:101E500063FE024B1B68C01A08BD00BF9001002042
:101E6000BFF34F8F0549064BCA6802F4E062134383
:101E7000CB60BFF34F8F00BFFDE700BF00ED00E078
:101E80000400FA054FF08053D3F83021082A06D118
:101E9000D3F83431052B02D8024AD05C70470020B9
:101EA000704700BF98530000024AD2F80034002B5C
:101EB000FBD0704700E0014010B54FF08053D3F8DD
:101EC0003021082A4ED14FF080420021C2F80C1177
:101ED000C2F81011C2F8381502F54042D3F80414C4
:101EE000C2F82015D3F80814C2F82415D3F80C143E
:101EF000C2F82815D3F81014C2F82C15D3F814140E
:101F0000C2F83015D3F81814C2F83415D3F81C14DD
:101F1000C2F84015D3F82014C2F84415D3F824149D
:101F2000C2F84815D3F82814C2F84C15D3F82C146D
:101F3000C2F85015D3F83014C2F85415D3F834143D
:101F4000C2F86015D3F83814C2F86415D3F83C14FD
:101F5000C2F86815D3F84014C2F86C15D3F84434AD
:101F6000C2F87035FFF78EFF18B13F4B3F4AC3F8F8
:101F70008C26FFF787FF18B13D4BFB22C3F81825CD
:101F8000FFF780FF70B14FF080414FF08053D1F8E0
:101F9000E42ED3F8583222F00F0203F00F0313435C
:101FA000C1F8E43EFFF76EFF20B1324B4FF40072F0
:101FB000C3F840264FF08053D3F83031082B1AD1A4
:101FC0004FF08043D3F80024D20744BF6FF00102E2
:101FD000C3F800244FF08053D3F83431052B02D8D6
:101FE000254AD35C3BB14FF01023D3F808224FF0C1
:101FF0008043C3F858254FF01021D1F80C32DB078D
:1020000014D51E480123C0F80435FFF74DFFD1F861
:102010000C3223F00103C1F80C32FFF745FF002317
:10202000C0F80435FFF740FFFFF71AFFD1F8003280
:10203000002B03DBD1F80432002B14DA0F49012303
:102040004FF01020C1F804351224FFF72DFFC0F81F
:102050000042FFF729FFC0F80442FFF725FF0023E5
:10206000C1F80435DEE710BD005000404881030090
:1020700000F00040009002409253000000E0014058
:1020800030B50468CCB1BFF35B8FB4FA84F3C3F10D
:102090001F03DBB201229A4024EA020250E8005FEB
:1020A000A54204D140E8002CBCF1000FF6D1BFF3EB
:1020B0005B8FE6D102480B7030BD0248FCE700BFE1
:1020C0000000AD0B0200AD0B10B50368CB40DB0781
:1020D00014D401238B400268BFF35B8F43EA0201F3
:1020E00050E8004F944204D140E8001CBCF1000FBE
:1020F000F6D1BFF35B8FEED1014810BD0148FCE77C
:102100000000AD0B0400AD0B014BC3F80405704794
:1021100000F00140F7B5044618B1012823D003B000
:10212000F0BD4FF080430222C3F808230122DA6099
:10213000C3F80401D3F80431064601238DF80730B3
:1021400042F210754FF08047D4B1012CE7D1D7F897
:102150000C3403F48033AEBB83B3012002F0EBFBFD
:10216000013DF4D12AE04FF080430022C3F8080378
:102170005860C3F80021D3F800310DF10706DCE701
:10218000D7F8183403F480333EB9002BC7D00120B0
:1021900002F0D1FB013DF3D1C1E7D7F8182402F0DA
:1021A00003023260002BBAD09DF80700012803D14A
:1021B00002F0C1FB013DC7D1012CB0D1054B00227B
:1021C0005A71ACE7D7F80C2402F001023270002BF0
:1021D000EAD1F3E714090020044B1A7922B901224D
:1021E00018609A800248704702487047140900201E
:1021F0000000AD0B0C00AD0B08B5074B1B682BB1F5
:102200000020FEF78DFC08B9FEF77CFC4FF0804300
:102210000022C3F8182508BD1409002010B510B11C
:10222000012843D010BD4FF08043D3F81814D3F8E1
:102230001824C80321D502F00303012B04D013B1E5
:102240000020FFF767FF00234FF080420220C2F812
:10225000183508224FF4827303F18043002119607E
:1022600002F180421C6801241460154A12680AB306
:102270004FF08043C3F80403D4E7D3F81424D10704
:10228000E1D5D3F81C249207DAD40D4A12681AB1AA
:102290000222C3F80423C5E7D3F80421002AFBD0A7
:1022A0000022C3F80421D3F80431BBE700224FF425
:1022B0008073D1E71A68002AFCD019601B68B1E767
:1022C0001409002010B54FF08043D3F800216AB103
:1022D0000022C3F80021D3F800210122C3F808230B
:1022E000114B587910B95A711B6898474FF08043C9
:1022F000D3F8042172B10022C3F80421D3F80421D9
:10230000D3F81824D3F81824920704D10122C3F873
:1023100018259A6010BD0222C3F80823024BBDE8BD
:1023200010401B680120184714090020036803F0BF
:102330001F025B09026004D0012B034818BF002074
:1023400070474FF0A040704700030050034A430914
:1023500000F01F00D35C1844C0B270479E530000C9
:1023600070B50546FFF7F2FF0C4C08300E4634F806
:102370001030DA0508D5C3F3432304EBC302284623
:1023800054F8333052689847A3682BB1E26831465D
:102390002846BDE87040184770BD00BF34000020DB
:1023A00008B5FFF7D3FF034B083033F81000400B9C
:1023B00008BD00BF3400002008B5FFF7C7FF034B7E
:1023C000083033F81000C0F3400008BD340000208E
:1023D00008B5FFF7BBFF034B083033F81000C0F31C
:1023E000401008BD34000020034611F0010010B574
:1023F000CCB20DD1A207C4F3400012D5094AD2F8DD
:1024000020055860C2F82005003818BF012008E0F8
:102410004FF0A041D1F820251A60C1F82025002AEC
:10242000E8D010BD0003005010B5FFF78FFF124A2F
:10243000083032F81030D9051CD5C3F3432123F4FA
:10244000F85322F8103002F10E04002034F8023F55
:1024500013F4807F03D0C3F3432399420AD00130A1
:102460003028F3D1002342F831300448BDE8104051
:10247000FFF72ABE10BD00BF34000020AC000020D2
:10248000F0B5054600200446012607468C420BD1D4
:10249000114BD3F87C2132B10022C3F87C21D3F850
:1024A0007C3140F00040F0BDE3B29B0003F5807248
:1024B0009B0806FA03F31D420BD002F1804202F59D
:1024C000C042D2F800C0BCF1000F02D01760126801
:1024D00018430134DAE700BF00600040F7B5064654
:1024E0000846FFF733FF194F00F108050C4637F88F
:1024F0001530DB0727D5304602F085FA2046FFF776
:1025000067FF40B12046FFF74BFF316800F5A2702E
:10251000002341F820302046FFF786FF002301A862
:1025200027F815300194FFF701FF019B00EB8300B2
:10253000074BD0F80027134043F00203C0F80037E0
:10254000044803B0F0BD0448FBE700BF340000209E
:10255000F0F8FCFF0000AD0B0400AD0B2DE9FF41CE
:10256000164680460846FFF7F1FE0D4631680446E0
:1025700009B32846FFF720FF18B12846FFF728FFC8
:1025800010BB0023CDE900338DF80E308DF80F30ED
:102590000DF10F020B4628460DF10E0102F0DBF99A
:1025A000474A04F1080132F8113023F0020343F0E6
:1025B000010322F81130736863B328461F78596805
:1025C000FFF7FAFE10B1D1B13E4826E03C4A04F1D3
:1025D000080032F8103023F02003DB04DB0C22F873
:1025E000103061B1032FEFD87168496891F800C0CD
:1025F000D8F80010A7B90CF5A27C41F82C70304A2D
:1026000004F1080132F8113023F01C0343EA870378
:1026100022F81130B3684BBB2B4804B0BDE8F08101
:1026200001EB8C0143EA4C33D1F810E52EF0030E98
:10263000C1F810E5D8F8001001EB8C0E43F0200330
:10264000DEF8101522F8103021F44F3121F44071DA
:10265000CEF810152902DEF8108501F47C5141EA0C
:10266000074141EA0801CEF81015C8E7D3E9006731
:102670002846FFF7D9FE002ECED0114DD5E9002314
:10268000964203D19F4201D1002209E00F480DF18B
:102690000F01FFF7F5FC0C4B9842BED19DF80F20BF
:1026A00045F8326005EBC20308345F6035F814303A
:1026B00043EA422343F4807325F81430ACE700BFAB
:1026C000340000200400AD0B0000AD0BAC00002076
:1026D0002DE9F0430C4685B08046204611461E4643
:1026E000FFF734FE054629B32046FFF765FE18B90B
:1026F0002046FFF76DFE18BB314F05F1080937F88A
:10270000193013F01C0F02D04B78012B18D0012385
:102710008DF80F300023CDE900134A1C8B1C204696
:102720000DF10F0102F017F937F8193043F00303E8
:1027300027F81930002E41D02046FFF73DFE18B98A
:10274000204805B0BDE8F08396F800C0D8F8003006
:102750001B4F0CF5A272002143F8221005F108026C
:1027600037F8121021F02001C904C90C27F8121003
:1027700075781DB3D8F80000B67800EB8C002D04F6
:10278000D0F8103523F4991323F4F853C0F810351A
:10279000230203F47C5305F440353605D0F810E5E8
:1027A0002B4306F4801641EA4C31334341F02001BB
:1027B00043EA0E0327F81210C0F810350248C0E7AC
:1027C000340000200400AD0B0000AD0B014BC3E949
:1027D000021270473400002010B508461446FFF777
:1027E000F7FD50B10846FFF7B1FD054B083033F84F
:1027F000103004485B0B237010BD0348FCE700BF9A
:10280000340000200000AD0B0400AD0B70B5164D78
:1028100095F8804006462CBB2146602205F1100049
:1028200002F0ACFA30682E6F21468E420ED10023A2
:10283000C0F87C31D0F87C3140F30730FEF762F904
:1028400001230A4885F88030AB6770BDCBB29B008E
:1028500003F580727C2B08BF845001F1010108BF91
:102860008358E2E70248F0E7340000200000AD0B97
:102870000C00AD0B034B93F88000003818BF01200B
:10288000704700BF340000200148FFF71DBC00BFA7
:10289000A80000200148FFF7F3BB00BFA8000020FC
:1028A00073B503681646D3F80423002AA8BF4FF077
:1028B00000420546A8BFC3F8042308460C46FFF7AC
:1028C00087FD00B30846FFF777FD0146D8B92046DB
:1028D000FFF766FD04B2A40004F580720346286881
:1028E0008150296882582144D1F8102542F0010214
:1028F000C1F810252EB12968012202FA03F3C1F8AC
:10290000043302B070BD2046FFF720FD0F4B0830A6
:1029100033F81030C3F38203042B12D0052B12D0EE
:1029200001A80194FFF702FD019AD0F81035D340B9
:1029300003F00103991C204602B0BDE8704002F08C
:1029400053B80321F7E70221F5E700BF3400002068
:102950002DE9F04F694BDFF8A881D3F80403D8F8CC
:102960007010C0B289B040F00040FFF789FD051E2D
:102970002FDAC24600235AF87C1F06A8CDE9063399
:10298000FFF732FD5F4B01930DF118094FF0000B7B
:10299000019A12F8013B0192DA0803F007031AF8D2
:1029A000022022FA03F3DA071CD409F10409BBF16F
:1029B000000F14D0D8F870104FF00040FFF760FD02
:1029C000D8F87C1006A8FFF70FFD0028DAD125F013
:1029D00000450124002D79D109B0BDE8F08F4FF0FA
:1029E000010BD5E7484B5B440293D9F8001000294E
:1029F000DBD0029B91FAA1F11C78B1FA81F141EA96
:102A000044142046FFF7A2FC0830059438F81070F3
:102A1000C808BB0819F80020039301F0070101233F
:102A200003FA01F122EA010209F8002005A8FFF7E4
:102A30007DFC059A039B02F5E072C7F3820650F80D
:102A400022205B073746C2F3014224D5204639468F
:102A5000D6B2FFF785FC05A80594FFF767FC059B38
:102A600003F5E07350F82330C3F301439E4207D1CE
:102A70000021204601F0B8FF3146204601F0B4FFA6
:102A800005A80594FFF752FC059B012202FA03F307
:102A9000C0F82035A9E7022A0CD10321204601F015
:102AA000A3FF06F00503012BEAD139462046FFF7C4
:102AB00057FCE5E702212046039201F095FF032E23
:102AC000F3D0039A032ADBD1022EEDE795FAA5F3A2
:102AD000B3FA83F304FA03F29B0003F1804303F596
:102AE000C04325EA0205D3F81005D3F81015C0F34A
:102AF0000520C1F30141FFF733FC6BE700600040A4
:102B000034000020AE530000AE53000001460148DF
:102B1000FFF7B6BAB800002038B5EFF311852023CF
:102B200083F31288BFF36F8F064B9C6801F0ABFFF5
:102B300085F31188BFF36F8F2046BDE83840FDF75D
:102B400065BF00BF1C09002038B5094B53F8204071
:102B5000013053F82050A54200D838BD636823B136
:102B6000204601F093FF0834F5E723689847FAE719
:102B7000D051000070B52B4B2B4C2C4D012286B050
:102B800003201A70FFF7E0FFFDF746FC01F09AFF03
:102B90000420FFF7D9FF2646AE4204F1300410D3DB
:102BA00000F04CFC204C224EAC4226D300F05AFCE4
:102BB000FDF7A6FA1F4A137B23F00103137306B037
:102BC00070BD54F80C3C059354F8103C049354F831
:102BD000143C039354F8183C029354F81C3C0193A2
:102BE00054F8203C009354E90A2354E90C0100F006
:102BF00013FA54F8303C5E65CDE7D4E90A23B3F10B
:102C0000FF3F08BFB2F1FF3F05D052EA0301206841
:102C100003D101F0C5FF3034C6E73146183000F06B
:102C2000D5FDF8E7270B00209050000090500000E1
:102C3000AD4C00002002002008B50348034A0021E3
:102C4000121A01F03BFF08BD800100202C0B002070
:102C500070B5002386B00122CDE90423134E144D34
:102C600001930F22CDE902321249142303FB0055D0
:102C700006EBC01604464FF4C07000FB04110E4B67
:102C800000954FF4A072304600F0C6F9737B0B4AF2
:102C9000EE6023F0040373734FF4046304FB033307
:102CA00013442C746B6006B070BD00BFA0010020FF
:102CB0001C09002080130020614B0000400B002005
:102CC000BFB50020FFF740FF2C4B83F308882C4D45
:102CD0002C4E6B692C4F43F400736B610024E0238E
:102CE00085F82230EC772C766C76AC7685F820402F
:102CF0006B6A43F4E0236B6285F82340FDF702FE24
:102D0000FDF7A4FF4FF0FF33AB62EB62FEF764F810
:102D1000FDF7C0FF1D4BB36040F201129A81C3E979
:102D20001844DC6601F09BFE0120FFF70DFF022036
:102D3000174DFFF709FF00F0B5FB164B75610593C2
:102D4000012315490094CDE903434FF480623B46CB
:102D5000CDE90144284600F05FF96A7B064622F07F
:102D6000040228466A7301F057FF2046FFF770FF00
:102D70003A4631462846FDF747FF00BF8013002042
:102D800000ED00E01C090020752B0000A0020020CF
:102D900020020020B05300000015002038B5064C7A
:102DA000064D0020AC4200D338BD204601F08BFE1A
:102DB0000028F9DB1C34F5E72C0100202C01002051
:102DC00073B50C46EFF31181202585F31288BFF30C
:102DD0006F8FC5685DB125602B68C360836901335F
:102DE0008361002081F31188BFF36F8F11E052EAF5
:102DF000030603D125606FF00B00F3E7CDE9002354
:102E00000246083000F066FA18B9034B9B685B690C
:102E1000236002B070BD00BF1C0900202DE9F34102
:102E2000044617461E46EFF31188202383F31288C9
:102E3000BFF36F8FC368334A7BB180689168884263
:102E400019D057EA060318D188F31188BFF36F8FA2
:102E50006FF00F0002B0BDE8F081916891F90E109B
:102E600021610133E3609368A36088F31188BFF3A5
:102E70006F8F0020EEE72169F2E791F90E1090F9CB
:102E80000E309942A8BF19466FF07E029142B8BF3A
:102E900011468B422DDD01F06EFE0546CDE9007630
:102EA00019482246414600F015FA0028E1D0EFF318
:102EB0001186202383F31288BFF36F8FA068D0B1EF
:102EC000236821699C420AD04BB193F90E30994294
:102ED000A8BF19466FF07E039942B8BF194601F0AA
:102EE0004AFE40B10848314600F064FA6FF00A002B
:102EF000B0E70025D2E7002DF4D186F31188BFF3A7
:102F00006F8FF3E71C090020280B002038B5836879
:102F1000044663B3194A926893422BD1C368012BCC
:102F200003D9013BC360002038BDEFF31185202396
:102F300083F31288BFF36F8F0169806801F01BFE75
:102F4000204601F0B7FEA06058B190F90E20226132
:102F50000022826701F060FE0948294600F02AFA43
:102F6000E1E7E06085F31188BFF36F8FDBE76FF077
:102F70001500D9E74FF0FF30D6E700BF1C0900204D
:102F8000280B002038B50446EFF31185202383F386
:102F90001288BFF36F8F01F08DFE48B10022826767
:102FA00001F03AFE29460848BDE8384000F002BA70
:102FB000D4E902329A4218BF0133A36085F3118825
:102FC000BFF36F8F38BD00BF280B002013B5EFF3A0
:102FD0001181202484F31288BFF36F8F846844B179
:102FE000013C846081F31188BFF36F8F002002B031
:102FF00010BD52EA030406D181F31188BFF36F8F2D
:103000006FF00F00F3E7CDE900230246014800F01E
:1030100061F9ECE7280B00202DE9F043073285B079
:1030200022F007020E461F461099017300F1580363
:103030007F32C0E916330446002322F03F02042108
:10304000836041733F2A0F98A073C4E90633E3738A
:1030500006F14009A2F1400805D883F31188BFF3B7
:103060006F8F084602DFB51829462046FDF7D2FAD1
:1030700007300E9B20F00700A066C4E91898029361
:103080000D9B01932D1A0C9B00932A463B4631461B
:103090002046FDF787FD00236365044B9B6803B161
:1030A000DB6EE366284605B0BDE8F0831C0900200E
:1030B00038B50D4D2B4653F8184F9C4200D004B93B
:1030C000EC68AB6838B95A7BD20604D1A26912B950
:1030D000DA897F2A05D89C4202D0204600F0BEFA49
:1030E00023466B6138BD00BF1C09002008B590F96C
:1030F0000D20437B002A014604DA03F07F0343736B
:1031000001F050FD044B9868431A58425841BDE8FD
:103110000840FFF7CDBF00BF1C09002070B490F934
:103120000D30427B002B29DBD30627D183692BBBD3
:10313000134962F07F0242730A4652F8184F9442D4
:1031400018BF2346CC6923B9C0E900242060C861B8
:103150000CE090F90E5093F90E60B5420AD0AE42E1
:1031600008DD5A68C0E900321060586070BC002069
:10317000FFF79EBF9C42E7D01B68E4E770BC704736
:103180001C0900202DE9F041002A427B0E460CBFAD
:1031900010210821114204460FD141EA0203D2094D
:1031A00018D1437308291BD00120FFF781FFBFF31B
:1031B0005F8F637B23F060036373274B9B68A3429D
:1031C00043D1EFF30583002B3FD13046BDE8F041FA
:1031D000FDF732BC03F07F03437301F0E3FCE1E74A
:1031E000A36813B1204601F0E5FC04F1180001F0DA
:1031F0009EFDA56D04F15807AF4211D04FF00008B5
:1032000075B1284601F0D6FC05F1180001F08FFDDC
:10321000C5F878802846FFF781FFA56DAF42EFD152
:103220000D4DAB689C42BFD1EFF30583002BBBD0A3
:103230000120FFF73DFF094BAB6040F201129A817C
:103240000022C3E91822DA66B1E786F31188BFF3DA
:103250006F8FBDE8F08100BF1C090020A002002094
:1032600070B590F90D20437B002A014604DA03F083
:103270007F03437301F096FC4B7B154A63F07F0399
:1032800010464B7350F8183FD469834208BF00239F
:1032900023B9C1E900042160D1610CE091F90E501D
:1032A00093F90E60B5420ED0AE420CDD5868C1E90C
:1032B0000030016059609068431A5842BDE8704080
:1032C0005841FFF7F5BE9C42E3D01B68E0E700BF22
:1032D0001C090020F8B5124B0C461146114A98689B
:1032E0001060DDE90676EFF31182202282F3128866
:1032F000BFF36F8F9D68284601F066FCB6F1FF3F73
:1033000008BFB7F1FF3F06D007493A46334605F1FB
:10331000180000F05BFA2046BDE8F840FDF78CBBD2
:103320001C0900203C090020AD4C0000F8B5044603
:10333000EFF31186202383F31288BFF36F8F437B53
:10334000DA0649B219D18569BDB903F07F03437329
:1033500001F028FC437B164A817363F07F034373BB
:10336000134653F8180F984218BF0546D0695DB947
:10337000C4E900300460D46111E0A173002086F339
:103380001188BFF36F8FF8BD95F90E70B9420BD05D
:103390008F4209DD6B68C4E900531C606C6001203A
:1033A000FFF786FE0120EAE7A842E1D02D68DEE7BC
:1033B0001C09002049B9EFF3058030B9054B5A6963
:1033C0009B689A4201D0FDF737BB81F31188BFF3A8
:1033D0006F8F70471C09002010B5EFF31184202275
:1033E00082F31288BFF36F8F427B510704D484F3BA
:1033F0001188BFF36F8F10BD22F004024273FFF7F4
:103400008DFE21460248BDE81040FFF7D3BF00BF44
:10341000280B0020034648B9EFF3058232B9064A6B
:1034200051699268914201D0FDF706BB83F3118880
:10343000BFF36F8F704700BF1C090020EFF31181AD
:10344000202383F31288BFF36F8F054B9A68D37BD9
:10345000013BD37381F31188BFF36F8F704700BFB7
:103460001C09002038B5EFF31185202484F312885D
:10347000BFF36F8F0A4B9A68D37B0133D37300205D
:10348000FFF716FE85F31188BFF36F8FEFF31180FE
:1034900084F31288BFF36F8FBDE83840FFF7BABFDF
:1034A0001C090020024B03F11802C3E906227047F1
:1034B0001C090020F8B5EFF31185202383F312884F
:1034C000BFF36F8F19498868437B03F07F03437311
:1034D00001F068FB8B685A7B084662F07F025A73E2
:1034E00050F8182FCC69824208BF002222B9C3E9E4
:1034F00000042360CB610CE093F90E6092F90E702A
:10350000BE420ED0B7420CDD5168C3E900210B600A
:1035100053600120FFF7CCFD2846BDE8F840FDF7D9
:103520008BBAA242E3D01268E0E700BF1C0900207A
:1035300050EA01032DE9F04105460E4603D1FFF79D
:10354000B9FF00202BE0831C71F1FF3329DB01F070
:1035500003FC2C18EFF31188202383F31288BFF3A8
:103560006F8F124F124BB8681860FFF7BFFDB86835
:1035700010492A463346183000F028F9BA68537BC0
:1035800043F0100353734046FDF756FA01F0E4FB95
:10359000201A63EB0303012873F10003D1DBBDE8BC
:1035A000F0816FF00104241AD4E700BF1C09002049
:1035B0003C090020AD4C0000B1F1FF3F08BFB0F165
:1035C000FF3F08B506D10A4B986801F034FB4FF075
:1035D000FF3008BDFFF7ACFF4FF47A7147F6FF7379
:1035E0000022C0FB0132D80B40EA4240F1E700BFA5
:1035F0001C090020014B9868704700BF1C0900207F
:10360000044BC01A044BC0105843044B01221A54F7
:10361000704700BF20030020ABAAAAAA280B0020F5
:10362000C3897F2B12D80A4B1B6863B1094B90F9F1
:103630000E201B689A4209DB437BDB0606D1064B52
:10364000C31A18BF012303F0010070470023FAE7F3
:103650004409002040090020A001002070B50E4B55
:103660000E4C1E7C06EB460304EBC30405462046C5
:1036700001F05DFB0A4B002228469A55FFF7D0FF68
:1036800048B1084B08491A68013A2046D317BDE8EB
:10369000704000F09BB870BD1C0900202003002082
:1036A000280B0020440900200136000038B5EFF354
:1036B0001185202383F31288BFF36F8F104B114ABB
:1036C0009C681068A04206D1FFF7C8FF85F31188F7
:1036D000BFF36F8F38BD00211B7C11600A4AD35C99
:1036E000002BF3D02046FFF79BFF0028EED0637B32
:1036F000DB0602D12046FFF7B3FD2046E4E700BF1A
:103700001C0900203C090020280B002008B50648B1
:10371000064A0749121A01F0D3F9BDE80840054AE4
:103720000549064801F0CCB9000000207C010020CA
:10373000C453000000000000C4530000000000203B
:10374000034B1B680BB9FEF781BB0020704700BF1D
:103750004809002030B570B10B4B5B6898420AD025
:10376000036843B1D3E90421D0E90445121941EBC0
:103770000501C3E90421D0E9003213605A60002337
:10378000C0E9003330BD00BFBC00002010B50E4BB7
:103790001C689C4204D1FFF7D3FF6FF0004010BDBE
:1037A000FFF7CEFF002CF8D0D4E904321B1A62EBED
:1037B000E072B3F1004F72F10001EEDA002AACBF03
:1037C00018460020EBE700BFBC000020B3F1FF3F2C
:1037D00008BFB2F1FF3FF8B504461D4616465ED05D
:1037E0008160EFF31187202383F31288BFF36F8F7B
:1037F000013275F1FF3324DA2E49D1E900206FF050
:1038000001039B1A4FF0FF3262EB00009E1B60EB3E
:103810000500012E70F1000301DA01260020C4E941
:103820000460254ED6F800C07568B44508BF4FF057
:10383000000CBCF1000F0DD1C4E900652C60746070
:103840001CE0FFF77DFF013645F10005361845EB1A
:10385000E070E4E7DCE90420D4E90431934271EB41
:10386000000E1DDAD21ADCF8043060EB0100CCE95E
:103870000420C4E900C31C60CCF804403368B342A0
:1038800009D09C4207D10D4B1C6824B9FFF77EFF7D
:103890002146FEF7ADFA87F31188BFF36F8FF8BDAD
:1038A0009B1A61EB0001AC45C4E90431C4D0DCF8DB
:1038B00000C0BEE738030020BC00002048090020FB
:1038C0002DE9F84FEFF3118C202383F31288BFF317
:1038D0006F8FDFF8B0A0DFF8B0902C4FC9F8000070
:1038E000DAF800000024504508BF00200025D7E981
:1038F0000021D9F80030E04678B3D0E9046C4FEAF3
:10390000E37EB3427EEB0C0B05DAF61A6CEB0E0489
:10391000C0E9046421E0B21841EBE671C0E9044556
:10392000C7E90021FFF716FF88F31188BFF36F8FF7
:1039300083689847EFF31188202383F31288BFF33D
:103940006F8FD9F80030DAF800009B1B5045C44651
:10395000C9F80030CBD1D7E900219A1841EBE373C5
:103960000024C7E90023C9F80040FFF70FFF2146F4
:10397000FEF73EFA88F31188BFF36F8FBDE8F84F6A
:10398000FFF794BEBC000020480900203803002047
:1039900010B5EFF31184202383F31288BFF36F8FE8
:1039A000FFF7CEFE054A0346D2E90001181841EBA5
:1039B000E37184F31188BFF36F8F10BD38030020CB
:1039C00010B50A4C23681BB101232360002010BDF1
:1039D00000F0EAF80028F7D00138062803D8044B95
:1039E00053F8200010BD034810BD00BF4C09002053
:1039F000E8510000FE8FFFFFBFF34F8F0549064BD4
:103A0000CA6802F4E0621343CB60BFF34F8F00BF7C
:103A1000FDE700BF00ED00E00400FA0510B4094B1B
:103A200009490A4C4FF0FE32C3F800244968C3F834
:103A30000424C3F80824C3F80C240023C4F8003578
:103A400010BC084700B00250C400002000A0025083
:103A5000D0E90012014BC3E900127047C4000020F6
:103A600010B5044650B1636813F0685F05D0064A8C
:103A7000934202D000232360626010BD034B0448D0
:103A80005B689847EFE700BF2C5F5CA9C40000208B
:103A900004520000C8B143680D4A934213D013F09A
:103AA000685F0ED0012350E8002F194640E8001C43
:103AB0009CF0000FF7D1012AF5D0BFF35F8F0020F3
:103AC000704704487047044870476FF4E0407047FF
:103AD0002C5F5CA9E98FFFFFEA8FFFFF80B143688D
:103AE000094A93420AD013F0685F05D0BFF35F8F95
:103AF0000023036018467047044870470448704725
:103B00006FF4E040704700BF2C5F5CA9E98FFFFFB6
:103B1000EA8FFFFF10B5044620B1044B636000221A
:103B2000226010BD0248FFF779FFF6E73A00003A3D
:103B30002C52000070B5D0E90023174C174D63607C
:103B4000D0E90230C4E9023022604868D1F800C0F0
:103B5000134BC3E900C0D5F81801D1F808C0C3F869
:103B600008C010F0685FD1F80CC00969C3F80CC038
:103B7000196110D00B49C5F8BC110023C5E94531C6
:103B800005F58A70C5F8B8319047236805F5DC70F3
:103B9000BDE87040184770BDE000002064090020B7
:103BA000CC0000202C5F5CA938B500F02FF820B1C4
:103BB000032400F063F8204638BD00F031F898B9CE
:103BC00000F0ACF898B90F4DD5F828391B0EF02B42
:103BD00008D1D5F8242A0C4B9A420AD0072400F0C9
:103BE00017F8E6E70624FAE70424204638BD002447
:103BF000F5E7012000F092F804460028F7D1C5F857
:103C00000C0AD8E700B002500000E0200020704706
:103C100000207047014BC3F8040A704700B00250FF
:103C200010B5114800F048F800B110BD0F4800F081
:103C300043F80028F9D10E4C204600F03DF800284A
:103C4000F3D10C4B0C481C6000F036F801460028FC
:103C5000EBD100F02DF8044608B1204610BD00F06D
:103C60003FF82046FAE700BF200100201C01002099
:103C700018010020100100201401002008B5084898
:103C800000F024F8074800F021F8074800F01EF87B
:103C9000064800F01BF8BDE8084000F00BB800BF74
:103CA000200100201C010020180100201401002028
:103CB00000207047704700BF08B5034B02681B68BF
:103CC00010689847002008BDE000002008B5034BAD
:103CD00002685B6810689847002008BDE00000207B
:103CE00070B5094C094D2069AB68984718B1084B6D
:103CF00008485B689847084AEB6820690021116012
:103D0000BDE87040184700BFCC000020E000002054
:103D1000C40000205052000060090020F8B51A4D80
:103D20001A4E0446B26828699047E8B9184F3B68B4
:103D30004CB1A3B1012B19D0013B3B602869F3685A
:103D400098470020F8BD43B9124A0121C2F8001576
:103D50001149D1F81029002AFBD101333B60F368E7
:103D6000286998470020F8BD0C48F8BD0A4AD2F8E7
:103D70001039002BFBD1074A6FF07E40C2F80035A6
:103D8000FFF748FF3B68D7E7CC000020E0000020A9
:103D90006009002000A0025000B00250E98FFFFF30
:103DA0000FB407B5064B04AA186852F8041B019219
:103DB00000F008F803B05DF804EB04B0704700BFF2
:103DC000F05000002DE9F04F8DB0436802938378E6
:103DD00015469A07804640F10D8100240E78002E8A
:103DE00000F00A81252E0BD04B1C03930134029B5B
:103DF0004146304698470028C0F2F6800399EDE727
:103E00004E788B1C252E0393F0D00027B946BB4675
:103E1000BBF11F0F38D8A6F12003102B0AD8DFE81A
:103E200003F02A0909300909092109090928092D7E
:103E300009091F00A6F13003092B33D92A2E37D1E7
:103E40001BF0400F55F8043B40F08280002BA7BFC9
:103E50004BF0200B9946C3F100094BF0280B01E011
:103E60004BF0010B039B13F8016B0393002ECFD192
:103E700030E04BF0020B4BF0040BF3E74BF0080B78
:103E8000F0E74BF0100BEDE7BBF17F0F19D8A6F16F
:103E90003003092BD2D81BF0400F03D00A2101FBBD
:103EA0000737DFE70A2101FB09394BF0200BD9E77F
:103EB0002E2E06D11BF0400F40F09E804BF0400BA1
:103EC000D0E76C2E31D02BD8682E36D06A2E3CD05D
:103ED0004C2E3AD0002F46F02003B8BF2BF0400202
:103EE000A3F16501BCBF1FFA82FB0027022901D99B
:103EF000612B2FD1073525F00705DFF8ACA2083577
:103F000007271BF0080F66D00AEB070B56465E45E5
:103F100063D1A4EB0A0A06EB0A02A9EB07096FE1D9
:103F2000742E9FD07A2E9DD0D4E71BF0800F18BF3F
:103F30004BF4007B4BF0800B94E71BF4807F18BFA1
:103F40004BF4007B4BF4807B8CE74BF4207B89E7C0
:103F50001F4687E7A6F16301122900F2F080DFE82F
:103F600011F013004F00EE00EE00EE00EE004F00E7
:103F7000EE00EE00EE00EE00EE00FE00E900EE00C6
:103F8000EE001B00EE00AF0055F8043B8DF8183032
:103F900001270DF1180AB4E755F804AB834BBAF1C9
:103FA000000F08BF9A461BF0400F14BF39464FF070
:103FB000FF31504600F0EAFE0746A2E7029B414669
:103FC0002020984700280FDB013EB742F6D34C442F
:103FD000A41BB14698E74E46F7E716F8010B029B83
:103FE00041469847002892DA98F8023043F00403DB
:103FF00088F802304FF0FF3420460DB0BDE8F08F56
:104000001BF0800F34D01BF4007F2CD0073525F037
:104010000705AA4669685AF8080B2BF01005002915
:10402000ADB237DA404261EB410145F480650DF1F4
:10403000180B0A235A4600F0B5FEA0EB0B030193C0
:104040006B0662D5019B25F001019F4289B240F3C6
:10405000A180002E00F0998015F0100240F09C80A5
:10406000BB460D4623E0AA465AF8040BC117D4E715
:10407000AA461BF4807F5AF8041B01D10846F5E7D5
:104080001BF4007F15BF48B208B241F3C01141F3E1
:10409000C031C2E750EA0103C9D11BF0400FC6D0BE
:1040A000002FC4D12BF0110295B2BB46019740F20C
:1040B000064115EA01021CBF0BF1010B00222CE0A6
:1040C0002BF010021FFA82FB0A231BF0800C49D050
:1040D0001BF400711DBF073525F00705AA46AA4647
:1040E0001ABF5AF8080B69685AF8040B50EA010520
:1040F00045D12BF016051BF0400FADB242D0002F7A
:1041000040D12BF0170295B2019715F0100248D05C
:10411000019B002E42D103F1010B29075AD4EB0772
:1041200006D5D9456FDD0199A9EB0B035F18CB4686
:104130005B4649E04BF0100B10237826C5E7782B3F
:1041400004D1C6F1780343F01003BEE7029B414659
:10415000252098470028FFF647AF023447E608239A
:104160000026B2E7AA461BF480715AF8040BBDD0B2
:104170001BF400711ABFC0B2614680B2B6E72BF0E3
:10418000060295B20DF1180B54E725F01105ADB2FA
:10419000BB468CE70D46B8E73B460D4603F1020BE4
:1041A000BBE7DDF804B082E7BC530000B553000064
:1041B000CDE904324146029B202098470028FFF6B3
:1041C00013AF049B059A01339945F1DCA4EB0B0175
:1041D000CC189B460AB3029B4146302098470028E2
:1041E000FFF602AF8EB901342744019B391B994277
:1041F00024DC1D465DBB019AA9EB0B092244554600
:104200001446914435E0019F92E70234414630461E
:10421000029B98470028E7DAE6E640F206410D42A5
:10422000E2D015F0020F14BF2B20202015F4806F70
:1042300004F10104414618BF2D20E9E7029B4146E5
:1042400030209847002804F10104CEDACCE606AB12
:10425000013D4146585D029B98470028CADAC3E6F3
:10426000029B414620209847002804F10104FFF6F4
:10427000BBAEA9EB0403002BF2DCBFE570478368FB
:1042800000EBC101B3F5004F2CBF51F8220031F80B
:104290001200704700EBC1018068B0F5004F2CBFE1
:1042A00041F8223021F81230704708B50122FFF79B
:1042B000E6FFD04008BD8368B3F5004F00EBC101B5
:1042C00008D34B681AB143F001034B60704723F0E9
:1042D0000103FAE74B881AB143F001034B807047A2
:1042E00023F00103FAE753000122FFF7D3BFB0F533
:1042F000004F34BF04230823481C0833A0EBD3002D
:10430000B0FA80F0C0F11F0070472DE9F0410D4672
:1043100086680446FFF7C9FFB6F5004F014601D392
:10432000012832D03046FFF7E2FF04EB80010E692E
:1043300096B9E368012282401343E36002220D61D3
:104340002B4629462046FFF7A5FF03222946204693
:10435000BDE8F041FFF79EBF022231462046FFF73D
:104360008EFF2946034607462046FFF793FF0322A8
:10437000334629462046FFF78DFF39462B46204617
:10438000FFF788FF02223146E1E7BDE8F081B2F590
:10439000802F2CBF08230423D21A2DE9F0418C185A
:1043A000CD1D25F0070524F00704641B0026E40852
:1043B00005602146AC60EE602046FFF798FF421D85
:1043C0009200013002F107074FEAD707A2F110026D
:1043D0003146B8BF324605F1100000F0CFFC3A4636
:1043E00031462846FFF77FFF33463246314628469E
:1043F000FFF750FFA4EB0708284631460122FFF7DC
:104400005AFF42463946FFF76EFF3B463246394671
:104410002846FFF73FFF21462846FFF764FF434643
:10442000324621462846FFF735FF2146284601221D
:10443000FFF741FF3946BDE8F041FFF766BF0020B6
:1044400070470FB407B504A951F8040B0191FBF7AD
:104450009DFE03B05DF804EB04B07047038B13F0CE
:10446000070305D10368002B0CBF00200320704711
:10447000022B05D1408BB0FA80F0400980007047D4
:10448000012B05D10368002B0CBF002005207047CD
:104490000020704710B50C4600B111B96FF015003F
:1044A00010BD081D00F093F80028F9D1A368032B74
:1044B000F6D9F3E72DE9F0410D4607461946281DC8
:1044C00090461E4600F094F8044638B13346424602
:1044D00029463846A446BDE8F0416047BDE8F08172
:1044E00010B4EFF31182202484F31288BFF36F8F8E
:1044F000416110BC0121FBF77BBE38B50C46054677
:1045000058B151B10B6843B14B6833B11C22002143
:1045100000F034FC2C61002038BD6FF01500FBE783
:1045200070B505460E46FFF7B5FF041E14DBEFF32A
:104530001182202383F31288BFF36F8F6B8B2C8B38
:104540004FF6FF718B4204F0070407D182F3118804
:10455000BFF36F8F6FF00A04204670BD022C0CD1A0
:1045600001336B8382F31188BFF36F8F00232246E0
:1045700031462846FFF79EFFEEE7062C14D8DFE809
:1045800004F004131313041A0400002333606B684F
:104590003BB9C5E90066ACB902212846FBF728FE05
:1045A000DAE71E606E60F6E782F31188BFF36F8F63
:1045B0006FF00404D0E782F31188BFF36F8F6FF0C0
:1045C0008504C9E782F31188BFF36F8FC4E7034600
:1045D00058B1426802F00302012A03D0032A04D131
:1045E000026812B10020986070476FF015007047A4
:1045F0004268816002F00302032A4FF00002034682
:104600000CBF006810465A6070477047FEE70128EB
:1046100001D1EFF30583FEF77FBA01460068FFF78B
:10462000F6BF08B5FBF7F2FFBDE80840FCF712B88B
:1046300000210120FFF7EBBF61B662B680F311885D
:10464000BFF36F8F704772B6002383F31188BFF3F7
:104650006F8FBFF34F8F30BF62B6BFF36F8F70475E
:1046600072B6002383F31188BFF36F8FBFF34F8FB0
:1046700020BF80F31188BFF36F8F62B67047202888
:1046800009D9B0F1004F08D80138B0FA80F0C0F174
:104690001F0040007047082070473E20704708B553
:1046A000FCF74EFC002008BD0369C9B20C2201FBD7
:1046B0000233186C00F00700704770B5C9B2036987
:1046C000EFF31185202484F31288BFF36F8F0C263B
:1046D00006FB0134246C14F0C00408D0A24206D0BA
:1046E00085F31188BFF36F8F4FF0FF3070BD06FB6D
:1046F000013301221A6485F31188BFF36F8F436879
:1047000003EBC1035B6898470020EFE78022FFF7C7
:10471000D4BFF8B5069F0469C9B2EFF3118620250E
:1047200085F31288BFF36F8F0C2505FB0144256CC0
:1047300005F0070CBCF1010F0CD1276486F311883A
:10474000BFF36F8FC4E90E23436853F831309847A5
:104750000020F8BD05F0C005AF4286F31188BFF315
:104760006F8F0CBF6FF077004FF0FF30F1E713B59C
:1047700080240094FFF7CDFF02B010BD10B4006993
:10478000CBB21C2403FB0400002110BC1047002006
:10479000FDF744BD002000F0DCB81046FEF7F2BB88
:1047A00043685B68D3F810350B600020704743689E
:1047B0005B6802EA010021EA0201C3F80805C3F8B8
:1047C0000C150020704743685B680020C3F808158B
:1047D000704743685B680020C3F80C157047436856
:1047E0005A68D2F8043521EA03000B40C2F80805E4
:1047F000C2F80C350020704710B503695868F8B14D
:10480000884219D19C6808685860A14200D198601C
:10481000002008602AB15A680A609A68596002B993
:104820009960002010E0814206D1086820609868F5
:104830008142EDD19C60EBE7044600680028F2D18C
:10484000002AE8D16FF0150010BD30B54368136041
:10485000057A446804EBC504A34202D36FF001005B
:1048600030BD5C798C4201D00833F0E70020F7E7D7
:1048700043681B68D3F88004C3F88004704742681B
:104880001368D3F8100150B1D269002012780A7071
:10489000C3F81001D3F8102101221A6070474FF0BD
:1048A000FF30704702680346D2F8580140B95B6890
:1048B000DB0706D4D2F82001003818BF012070476A
:1048C0000120704743681B68D3F80423D20517D52D
:1048D000D3F82021A2B1EFF31182202181F31288B5
:1048E000BFF36F8FD3F8201131B10021C3F820112D
:1048F000D3F820110121D96082F31188BFF36F8FA3
:10490000D3F85831704700F150039B009BB203F17C
:10491000804303F5883300221A601B687047FFF755
:104920004FB808B5FBF786FDFBF75AFEBDE8084017
:10493000FFF746B8004700F08EB8C00000F1804095
:1049400000F5F830C0F81015C0F814257047FEF7D0
:10495000DDB8FDF7DFBBF7B5019001A8DDE9084739
:1049600016461D46FDF7E2FC019BB6F1000C18BF90
:104970004FF0010C00EB83000B1E18BF0123002D2C
:1049800043EA4C0314BF4FF00C0C4FF0000C002C0A
:1049900043EA0C0314BF4FF4E06C4FF0000C002FFF
:1049A00043EA0C03D0F8002714BF4FF4403C4FF00B
:1049B000000C43EA0C0322EA030301B109780EB1AB
:1049C0003678760019430DB12D78AD0031430CB126
:1049D0002478240229430FB13F783F040C433C4321
:1049E000C0F8004703B0F0BD1FB50DF10F030193F0
:1049F00000238DF80F1000931A461946FFF7ABFFFE
:104A000005B05DF804FB38B5054608460C46FDF7D1
:104A1000DFFCB0B10846FDF7CFFC90B90846FDF7C2
:104A2000BFFC2A6801238340C2F808332A6803B216
:104A300002EB8303D3F8102522F00302C3F81025FC
:104A400038BD20460021BDE83840FFF7CDBFFDF757
:104A500045BDFFF7D8BF08B1FCF7BABA7047704739
:104A600040B1C368587810F001001EBF1878B0FA42
:104A700080F040097047EFF31183202383F31288FD
:104A8000BFF36F8FFEE708B5FFF7F5FF10B5D0E96C
:104A9000003433B90020E268537843F001035370C7
:104AA00010BD204698470028F4D00028B8BF4042E7
:104AB000E368FF28A8BFFF201870ECE700F05EB99C
:104AC00000F04EB970474169836843EA010212F071
:104AD00003020FD1C2600269013A01FB023382680E
:104AE0009A4201D900207047C2681A604269C360C7
:104AF0009B1AF4E76FF01500704710B5C0E9043257
:104B00000023816083610446FFF7DDFF0028A8BF12
:104B1000C4E9004410BDF8B504460D46EFF3118614
:104B2000202383F31288BFF36F8FC7686FB900F03B
:104B3000C1F850B18767456100F06EF8314604F165
:104B40000800BDE8F840FEF735BCE3682B60A369B8
:104B5000E560013BA36186F31188BFF36F8FF8BD59
:104B600008B52024EFF3118384F31288BFF36F8F0D
:104B7000FFF769FDF6E790F90E308B4201D0FEF7A2
:104B8000D5BB0020704703460020C3E90200C3E9FB
:104B900000337047EFF30580003818BF01207047DD
:104BA000FEF71ABCD0E9003213605A600023C0E956
:104BB0000033704708B5FFF7F5FF437B23F002038E
:104BC00043730023836008BD38B504460D46FEF7E5
:104BD0008DFA637B43F002036373E5B1A5602B6834
:104BE0009D4209D16B68C4E900531C606C6012E0FF
:104BF0006A689A42F6D01B68002BF3D094F90E2015
:104C000093F90E108A42F3D09142F1DD5A68C4E95B
:104C1000003214605C6038BD10B5EFF311842023BE
:104C200083F31288BFF36F8FFEF778FA84F311884D
:104C3000BFF36F8F10BD10B50446183000F077F841
:104C4000EFF31181202383F31288BFF36F8F627B10
:104C500012F0100204D081F31188BFF36F8F10BDE2
:104C60002046BDE81040FEF78DBA38B50446EFF394
:104C70001185202383F31288BFF36F8F437B13F0DA
:104C8000280F0BD183680BB1FFF794FF637B51B9F9
:104C900003F0FB0363732046FEF740FA85F31188A7
:104CA000BFF36F8F38BD03F0EB03F3E70121183832
:104CB000FFF7DBBF38B5EFF31185202383F31288AC
:104CC000BFF36F8F0468A0420DD034B12046FFF7C8
:104CD00071FF04F1180000F02AF885F31188BFF382
:104CE0006F8F204638BD0024F7E7EFF311812022B3
:104CF00082F31288BFF36F8F027BD2070CD581F34A
:104D00001188BFF36F8F002383F31188BFF36F8F78
:104D10000423184602DF7047437B1B0704D581F349
:104D20001188BFF36F8F70470122FEF72BBA10B5C1
:104D3000EFF31184202282F31288BFF36F8F036890
:104D40003BB1FEF707FD002084F31188BFF36F8F9E
:104D500010BD6FF01500F7E708B5FEF719FE08BDA6
:104D60000A44914200F1FF3300D1704710B511F8A9
:104D7000014B03F8014F9142F9D110BD02440346A3
:104D8000934200D1704703F8011BF9E710B50246C2
:104D900001448A42134603D01C780132002CF8D11A
:104DA000181A10BDF0B5C3F137070446FFB203F07F
:104DB0001F031046082BE6B233D0102B3ED06508F7
:104DC000A40844EA817445EAC1752D194FEA91029D
:104DD00042EB5102290941EA02716D1842EB1212AD
:104DE000290A41EA02616D1842EB1222290C41EABC
:104DF00002416D1842EB1242AD1842F10002EC087C
:104E000044EA4274D10804EB8402A6EB4205EDB2F9
:104E1000092D0CD90134A5F10A0541F10001EDB2CB
:104E200012E0E40844EA417406F00705C908303589
:104E300054EA010200F8015BBCD1F0BD240944EA48
:104E4000017406F00F050909092D84BFED19EDB2B3
:104E5000EDE7000001480068704700005C08002092
:104E60008D0F00000000000009110000C04E00007E
:104E70009D2D000000000000C1140000D44E000071
:104E8000C1140000E84E0000E50F00000000000023
:104E90001F4900000000000025190000FC4E000022
:104EA00071130000000000008D1C000000000000D5
:104EB000690F00000000000023490000000000000E
:104EC0005153000000510000105100002401002047
:104ED00090080020605300002C5100005C5100003D
:104EE00026010020E40800206E5300004451000019
:104EF0005C51000028010020F008002084530000CD
:104F000080510000C45100002A010020FC0800204C
:104F1000C5220000354900000000000031460000B5
:104F2000FC4E0000C54800000000000031460000B3
:104F30000000000031460000000000003146000083
:104F400051290000354900000000000031460000F2
:104F50000000000031460000000000003146000063
:104F60000000000031460000000000003146000053
:104F70000000000031460000000000003146000043
:104F80000000000031460000000000003146000033
:104F90000000000031460000000000001D1D000060
:104FA0000000000031460000000000003146000013
:104FB0000000000031460000000000003146000003
:104FC00000000000314600000000000031460000F3
:104FD00000000000314600000000000031460000E3
:104FE00000000000314600000000000031460000D3
:104FF00000000000314600000000000031460000C3
:1050000000000000314600000000000031460000B2
:1050100000000000314600000000000031460000A2
:105020000000000031460000000000003146000092
:105030000000000031460000000000003146000082
:105040000000000031460000000000003146000072
:105050000000000031460000000000003146000062
:105060000000000031460000000000003146000052
:105070000000000031460000000000003146000042
:105080000000000031460000000000003146000032
:105090000338FDD870470000000000000D460000F6
:1050A0001C000020140000200C0000200000000064
:1050B000040000204D05000041040000950400009C
:1050C000F5040000000000200000000000000B06B6
:1050D00002000000D8500000000000003C53000017
:1050E00026000207000000204453000022000B119C
:1050F000240000209110000061100000000000005A
:10510000E1110000D51000008F4700009547000016
:10511000611100000D4700006F4700000000000013
:10512000A94600000000000000000000FFFF000092
:10513000000300500000000001000000006000407B
:1051400000000000FFFFFFFF000000500000000013
:105150000000000000600040000000005515000045
:10516000A1470000AF470000C7470000D347000039
:10517000DF470000C1130000F947000000000000F5
:10518000002000400100000000000000A0510000CD
:105190000000D60100000000260B0020250B002097
:1051A00000200040AC51000001000000B45100009C
:1051B000040000000D000000110000020F060001B5
:1051C000140600037F4800007118000071480000B9
:1051D000604E0000604E0000A84E0000B04E00007F
:1051E000C04E0000C04E0000FF8FFFFFFF8FFFFF8B
:1051F000FE8FFFFFFE8FFFFFFD8FFFFFFC8FFFFF86
:10520000FC8FFFFF6D757465785F6672656520635E
:10521000616C6C65642077697468204E554C4C2035
:10522000706172616D6574657200000043616E2784
:105230007420696E697469616C697A65206D757432
:1052400065782C20776173204E554C4C0D0A000078
:10525000436F756C64206E6F74206C6F636B20708D
:105260006F7765722073617665206D75746578005F
:105270004F4E004F4646004C4544207374617465A0
:105280003A2025730A002A2A2A20426F6F74696E19
:1052900067206E524620436F6E6E656374205344E0
:1052A0004B2076322E392E302D3737383762323652
:1052B0003439383430202A2A2A0A002A2A2A20554A
:1052C00073696E67205A6570687972204F53207633
:1052D000332E372E39392D316638663364633239CF
:1052E000313432202A2A2A0A006D757465785F6984
:1052F0006E69742063616C6C6564207769746820E2
:105300004E554C4C20706172616D6574657200433E
:105310006F756C64206E6F7420616C6C6F63617468
:1053200065206D75746578206265666F72652069A9
:105330006E697469616C697A696E6700464C4153A5
:10534000485F30005352414D5F30000000010000C3
:1053500000636C6F636B403430303030303030007D
:105360006770696F403530303030333030006770EF
:10537000696F40353030303030303000000102038A
:1053800004050607756172744034303030323030B5
:1053900030000000000000010100000000000020BB
:1053A000303030303030303030303030303000015C
:1053B0006D61696E00286E756C6C29002A666C6FD1
:1053C00061742A003F440000400100203A000000C0
:1053D000540100203A0000002C0100203A00000097
:1053E000680100203A000000000000009F46000015
:1053F00000000000000000000000000000000000AD
:10540000000000000000000000000000000000009C
:10541000000000000000000000000000000000008C
:10542000000000000000000000000000000000007C
:10543000000000000000000000000000000000006C
:10544000000000000000000000000000000000005C
:10545000000000000000000000000000000000004C
:10546000000000000000000008000000FF00000035
:10547000000000000300000000000000FFFF0F001C
:10548000BC000020BC00002000000000F939000032
:105490000801002000010020F800002000000000AA
:1054A000F0000020153B0000613A0000953A000032
:1054B000DD3A0000500900203A00003A540900206B
:1054C0003A00003A580900203A00003A5C090020EE
:1054D0003A00003A18010020DC000020D40000202F
:1054E000D0000020CC0000200000000000000000E0
:1054F0002C0100202C010020000000000000000012
:105500000E000000400100204001002000000000CB
:10551000000000000E000000540100205401002093
:1055200000000000000000000E00000068010020E4
:105530006801002000000000000000000E000000D4
:0455400015E015E07D
:00000001FF
